:100000000C9446000C9463000C9463000C94630001
:100010000C9463000C9463000C9463000C946300D4
:100020000C9463000C9463000C9463000C946300C4
:100030000C9463000C9463000C9463000C946300B4
:100040000C94AE020C9463000C94E3020C94340301
:100050000C9463000C9463000C9463000C94630094
:100060000C9463000C94C1040C9463000C94630022
:100070000C9463000C94AA040C940B030C945B0383
:100080000C9463000C9463000C94630011241FBE55
:10009000CFEFD0E1DEBFCDBF12E0A0E0B1E0E6EEF1
:1000A000F5E100E00BBF02C007900D92AA32B10744
:1000B000D9F714E0AAE2B2E001C01D92AC39B10751
:1000C000E1F70C949D000C940000CF92DF92EF9228
:1000D000FF920F931F93CF93DF936C018AB59BB56B
:1000E0007C01002711278AE0C816D104E8F0D60168
:1000F000CC27DD27AE15BF05C007D107A9F088B50D
:1001000099B59C0144275527BD01CE010E94810A63
:10011000DC01CB01BC01CD01A80197010E94A00A1E
:10012000DBBCCABC39BD28BDDF91CF911F910F91B7
:10013000FF90EF90DF90CF900895CBEFD0E1DEBF3E
:10014000CDBF19821A821B821C82222433240E9472
:100150005A0468EC73E083EE93E00E94540580E05B
:1001600091E00E94260686E091E00E94260680E04B
:1001700091E00E942606EFE2F2E0A0E0B0E085E028
:10018000182E0E94C80A8091310290913202009785
:1001900019F08F5F9F4F31F481E090E0909332022D
:1001A0008093310280913102909132029F938F931C
:1001B00080E391E09F938F930E9411068091330218
:1001C00099279F938F9381E491E09F938F930E944F
:1001D00011068091330283BD8DB79EB708960FB686
:1001E000F8949EBF0FBE8DBF8091650090E1892776
:1001F0008093650080E00E94A302482E552481E090
:100200000E94A302682E7724620136E0CC0CDD1C2C
:100210003A95E1F7AFE3B0E0CA0EDB1EC301AA27AF
:10022000BB274601AA24BB24BC01CD01A501940132
:100230000E94810ADC01CB01BC01CD012FEF30E02F
:1002400040E050E00E94A00A79018A01DBBCCABCF0
:1002500039BD28BD85B39927969587958170907093
:100260009F938F93C801B70124E630E040E050E04F
:100270000E94810ADC01CB01BC01CD01A5019401E2
:100280000E94A00A5F934F933F932F931F930F9366
:10029000FF92EF92DF92CF927F926F925F924F9296
:1002A000F101EE5AFE4F8081992787FD90959F932B
:1002B0008F9387E591E09F938F930E941106089496
:1002C000211C311CB3E02B223324809151049091E6
:1002D0005004891BEDB7FEB774960FB6F894FEBFB5
:1002E0000FBEEDBF853008F479C0F89480915104B9
:1002F000E82FFF273597EF70F070EE0FFF1FEE0F1E
:10030000FF1FE05BFB4F2281338144815581809147
:100310005104E82FFF273197EF70F070EE0FFF1FA9
:10032000EE0FFF1FE05BFB4FE280F380048115813D
:10033000789457016801A21AB30AC40AD50AC1F118
:1003400089819A81AB81BC81E816F9060A071B07EF
:1003500049F483E991E09F938F930E9411060F90D7
:100360000F9038C080913102909132029C01442755
:100370005527C601B5010E94810A9B01AC0160E0CE
:1003800078E38CE99CE10E94A00A5F934F933F932E
:100390002F9383EA91E09F938F930E941106ADB74C
:1003A000BEB716960FB6F894BEBF0FBEADBF12C053
:1003B000DF92CF92BF92AF9283EB91E09F938F93A6
:1003C0000E941106EDB7FEB736960FB6F894FEBF41
:1003D0000FBEEDBFE982FA820B831C8308E110E0B7
:1003E0000E94D7029091CF038091CE03981709F411
:1003F000A5C080919204909193040E949B05992737
:1004000087FD90950E94C20A282F332727FD30953B
:100410002436310509F455C02536310524F4233638
:10042000310551F08BC02536310509F450C02F3607
:10043000310509F452C082C080913102909132029C
:100440009F938F9384EC91E09F938F930E9411066A
:1004500086ED91E09F938F930E9411064091920444
:100460005091930464E170E084E392E00E94DE0521
:100470002DB73EB72A5F3F4F0FB6F8943EBF0FBE71
:100480002DBF892B09F45AC084E392E00E941F0516
:100490009093320280933102009719F08F5F9F4F43
:1004A00031F481E090E09093320280933102A2E037
:1004B000B0E080913102909132020C010E94D90A81
:1004C0003DC08DEE91E00E942606A99837C08CEFC2
:1004D00091E00E942606A99A31C0809133029927A3
:1004E0009F938F938AE092E09F938F930E941106CF
:1004F00086E192E09F938F930E94110640919204AF
:100500005091930464E170E084E392E00E94DE0580
:10051000ADB7BEB716960FB6F894BEBF0FBEADBF4F
:10052000892B61F084E392E00E941F0580933302DF
:1005300083BDA4E0B0E0082E0E94CD0A0150104017
:1005400017FF4ECF51CE97B1907C982B906297B900
:10055000369A3699FECF85B1992708951F920F924A
:100560000FB60F9211248F939F9380912C028F5F6F
:1005700080932C028A3058F010922C0280912A022B
:1005800090912B02019690932B0280932A0286E091
:1005900082BF9F918F910F900FBE0F901F90189563
:1005A00084E083BF12BE81E087BF789408952091D4
:1005B0002A0230912B0280912A0290912B028217FD
:1005C0009307C9F308951F920F920FB60F9211244B
:1005D0002F938F939F93EF93FF932CB18091CF0331
:1005E0009091CE03891B803861F08091CF03E82F72
:1005F000FF27EF77F070E253FC4F22838F5F8093E9
:10060000CF03FF91EF919F918F912F910F900FBE8C
:100610000F901F9018951F920F920FB60F921124F2
:100620002F938F939F93EF93FF9320919C00809142
:10063000490290914802891B803861F080914902FB
:10064000E82FFF27EF77F070E85BFD4F22838F5F85
:1006500080934902FF91EF919F918F912F910F907D
:100660000FBE0F901F9018951F920F920FB60F920A
:1006700011248F939F93EF93FF939091CB028091DE
:10068000CA02981711F455980DC08091CA02E82F3C
:10069000FF27EF77F070E653FD4F8F5F8093CA021C
:1006A00082818CB9FF91EF919F918F910F900FBE36
:1006B0000F901F9018951F920F920FB60F92112452
:1006C0008F939F93EF93FF9390914D0380914C03F1
:1006D000981731F480919A008F7D80939A000EC014
:1006E00080914C03E82FFF27EF77F070E45BFC4F1D
:1006F0008F5F80934C03828180939C00FF91EF91E8
:100700009F918F910F900FBE0F901F901895CF93D0
:10071000C82F8A3019F48DE00E9487038091CB02A4
:100720009091CA02891B8038C9F38091CB02E82FCF
:10073000FF27EF77F070E653FD4FC2838F5F809302
:10074000CB02559A80E090E0CF910895CF93DF934C
:100750009091CF038091CE039817D1F38091CE036F
:10076000E82FFF27EF77F070E253FC4F9281C92FFB
:10077000DD278F5F8093CE03CD30D10511F4CAE021
:10078000D0E08C2F0E948703CE01DF91CF91089596
:100790000E94A603089590914902809148029817FB
:1007A000D1F380914802E82FFF27EF77F070E85BE4
:1007B000FD4F92818F5F80934802892F992708957A
:1007C0000E94CB0308950E9487030895CF93C82FFA
:1007D0008A3019F48DE00E94E60380914D039091D8
:1007E0004C03891B8038C9F380914D03E82FFF2704
:1007F000EF77F070E45BFC4FC2838F5F80934D0313
:1008000080919A00806280939A0080E090E0CF917E
:1008100008950E94E6030895CF93DF93EC01888149
:10082000882361F088818A3019F48DE00E94870363
:1008300089910E94870388818823A1F7DF91CF9156
:100840000895CF93DF93EC018881882361F088813C
:100850008A3019F48DE00E94E60389910E94E60334
:1008600088818823A1F7DF91CF9108950F931F937B
:10087000CF93C62F8C01662339F0F80181918F0147
:100880000E948703C150C9F7CF911F910F9108951E
:100890000F931F93CF93C62F8C01662339F0F80175
:1008A00081918F010E948703C150C9F7CF911F9199
:1008B0000F9108959FEF9BBB1ABA98BB80ED87BB41
:1008C0008DEF85BB82E084BB92BB11BA93B912B89D
:1008D00010926200109261009093650088E180930D
:1008E000640010BE1092900029E129B91BB898E964
:1008F0009AB98EE080939500109298002093990009
:1009000010929B0090939A0080939D0087EC86B98B
:1009100080E487B986B1877C11F03699FECF0E94BA
:10092000D00280E094E09BBD8ABD80E092E099BD5A
:1009300088BD83E28FBD81E18EBD10927A008FEF7A
:1009400083BD8DE185BD82E880938A0084E2809337
:100950007D0008951F920F920FB60F9211248F936E
:100960009F9380912D0290912E02019690932E02DA
:1009700080932D029F918F910F900FBE0F901F902B
:1009800018951F920F920FB60F9211242F933F9339
:100990004F935F938F939F93AF93BF93CF93DF93C7
:1009A000EF93FF938091880090918900DC01C091C2
:1009B0002D02D0912E028091650098E089278093C6
:1009C00065008091510490915004891B803198F00A
:1009D00080915004E82FFF27EF70F070EE0FFF1F9B
:1009E000EE0FFF1FE05BFB4F228133814481558175
:1009F0008F5F8093500480915104E82FFF27EF70A0
:100A0000F070EE0FFF1FEE0FFF1FE05BFB4FA283A6
:100A1000B383C483D5838F5F80935104FF91EF919B
:100A2000DF91CF91BF91AF919F918F915F914F9146
:100A30003F912F910F900FBE0F901F901895FC01C2
:100A400088279927E89421912223F1F02032D9F3C5
:100A50002930C9F32A30B9F32C30A9F32D3099F39A
:100A6000263789F32B3219F02D3221F46894219125
:100A7000222351F0203344F02A3334F420530E94CF
:100A80004C05820F911DF3CF8115910521F01EF4C5
:100A900080959095019608957AE0979F902D879F75
:100AA000802D910D112408950F931F93CF93DF9301
:100AB0008C01EB01009711F4672BC1F16EE070E03F
:100AC00081E090E00E941909FC01892B71F180E816
:100AD0008383209771F0D387C28781E883838091D5
:100AE000920490919304892B21F4F0939304E09362
:100AF000920401151105C9F0118700878381826076
:100B000083838091940490919504892B71F4F093E0
:100B10009504E09394048091960490919704892B16
:100B200021F4F0939704E0939604CF01DF91CF91E5
:100B30001F910F910895CF93DF93EC014B81842F88
:100B4000992780FF2EC086FF09C04F7B4B838E8183
:100B50009F8101969F838E838A812CC082FF11C062
:100B6000E881F9818081282F332727FD30952115D1
:100B7000310519F440624B8314C03196F983E88340
:100B800013C0EA85FB85CE0109959C0197FF0CC037
:100B90008B8199272F5F3F4F11F4806101C08062E4
:100BA0008B838FEF9FEF07C08E819F8101969F837C
:100BB0008E83822F9927DF91CF910895CF92DF9274
:100BC000EF92FF920F931F93CF93DF936C01EB0192
:100BD0007A01FA01838180FF03C0161617061CF004
:100BE00080E090E015C0219786011C161D066CF46C
:100BF000C7010E949B05FFEF8F3F9F0789F3F80114
:100C000081938F0121970A9781F7F8011082C6011D
:100C1000DF91CF911F910F91FF90EF90DF90CF90D8
:100C20000895CF93DF93CDB7DEB7E5E0F0E0EC0FAA
:100C3000FD1F81919191AF01BC018091940490912D
:100C400095040E945C06DF91CF9108950F931F9346
:100C5000CF93DF93EC0100E010E0E0919404F09179
:100C60009504838181FD03C08FEF9FEF20C08991A0
:100C7000882371F0E0919404F091950420853185EA
:100C8000BF01F9010995892B91F30FEF1FEFEFCF0A
:100C9000E0919404F091950420853185BF018AE0AC
:100CA000F9010995892B11F00FEF1FEFC801DF91B2
:100CB000CF911F910F9108952F923F924F925F9283
:100CC0006F927F928F929F92AF92BF92CF92DF925C
:100CD000EF92FF920F931F93CF93DF93CDB7DEB7C1
:100CE00062970FB6F894DEBF0FBECDBFEE24FF248F
:100CF00087011C017E876D872A01CC24DD24FC013D
:100D0000D782C682838181FD68C28FEF9FEF78C250
:100D10008D859E8501969E878D87C0FE4BC28F85EF
:100D200080538A30D0F49F85903339F4662029F4BB
:100D3000C3FC03C0E0E0F1E08DC08AE0689E602C57
:100D40001124FF856F0E20ED620E67FE02C05FE783
:100D5000652EC3FC42C2762C40C2C3FE04C066208E
:100D600011F441E0642EEF858E2F992787FD909531
:100D7000883691058CF5853691050CF06EC083356B
:100D8000910509F493C084359105CCF48B3291051B
:100D900009F449C08C3291054CF48032910509F474
:100DA00046C08332910509F44AC0FEC18D329105D7
:100DB00009F440C08E32910509F444C0F5C1833670
:100DC000910509F450C0843691050CF08AC088352D
:100DD000910509F4BCC0E8C18037910509F4B1C0A0
:100DE0008137910584F48C36910591F18D3691050A
:100DF0002CF48936910509F474C0D6C18F3691055B
:100E000009F49CC0D1C18537910509F4A2C0863789
:100E1000910524F48337910571F1C6C18837910596
:100E200009F495C0C1C180E190E0C82AD92AE0E266
:100E3000F0E010C080E890E0C82AD92ACEC1E0E4F2
:100E4000F0E008C088E090E0C82AD92A6624C5C12D
:100E5000E4E0F0E0CE2ADF2AC0C13FE3E32E7A943B
:100E6000F3E6FF873CC1F20182E090E0480E591E94
:100E7000E0807A9434C1F20182E090E0480E591E7D
:100E8000A081B1817D01C3FE09C0862D992787FD10
:100E90009095BC01CD010E94490A1FC0FD0101903F
:100EA0000020E9F73197EA1BE88B18C0F20182E0D5
:100EB00090E0480E591E0190F081E02D7F01C3FEA5
:100EC00009C0862D992787FD9095BC01CF010E940E
:100ED000340A03C0CF010E942B0A888B9889791AA3
:100EE000FEC0C2FE0AC0F20184E090E0480E591E26
:100EF00020813181428153810CC0F20182E090E077
:100F0000480E591E808191819C01442737FD4095F0
:100F1000542F79018A0157FF0CC0E2E0F0E0CE2A9D
:100F2000DF2A10950095F094E094E11CF11C011D5E
:100F3000111D8FEB9FEFC822D92227C098E0988B14
:100F400008C0E0E4F0E0CE2ADF2AF8E7FF8720E1DE
:100F5000288BC2FE0AC0F20184E090E0480E591EC0
:100F600020813181428153810AC0F20182E090E008
:100F7000480E591E808191819C0144275527790193
:100F80008A01EFECFFEFCE22DF22CE0101969A8B91
:100F9000898B9889892E9924AA24BB24C801B7017A
:100FA000A50194010E94A00ADC01CB01E989FA891C
:100FB00080838A3024F0FF858F0F815201C0805DCD
:100FC000E989FA898193FA8BE98BC801B701A501F8
:100FD00094010E94A00A79018A0121153105410579
:100FE0005105E1F6E98881E090E08C0F9D1FE81A39
:100FF000C60182739070892B09F07A94C6FE0DC0E9
:10100000872D992787FD9095E889E03121F42EEF0F
:10101000722E780E02C0782E7A94C3FE0FC0262D51
:10102000332727FD30958E2D9927821793072CF0B3
:1010300087EF9FEFC822D92201C06E18C3FE02C0FD
:10104000761801C07E18C60180789170892B51F402
:10105000872D7A94181634F4B10180E290E00E9452
:10106000540AF6CFC1FE04C0B1018DE290E00BC07E
:10107000C4FE04C0B1018BE290E005C0C5FE05C00E
:10108000B10180E290E00E94540AC6FE10C0B10196
:1010900080E390E00E94540A9889903141F4B101B4
:1010A000EF858E2F992787FD90950E94540AD0FED8
:1010B0000AC0872D7A94181634F4B10180E390E0C9
:1010C0000E94540AF6CFC3FE0AC0862D6A941816F1
:1010D00034F4B10180E390E00E94540AF6CF90E826
:1010E000B92EBC2051F4872D7A94181634F4B1012E
:1010F00080E290E00E94540AF6CFFF85F33641F477
:101100008E2DB101992787FD90950E94540A40C009
:101110002F852337B1F488898150888B8F3FC1F1A7
:10112000F70180810894E11CF11CB101992787FD2A
:1011300090950E94540A98899150988B9F3F81F70F
:1011400027C0EF85E33579F4F889F150F88BFF3F3C
:10115000F9F0F7018491B10199270E94540A08948B
:10116000E11CF11CF1CF6E010894C11CD11C8989CE
:101170009A898C159D0561F0E989FA898291FA8B2B
:10118000E98BB101992787FD90950E94540AEFCF12
:10119000BB2069F0872D7A9418164CF4B10180E2D7
:1011A00090E00E94540AF6CFB1010E94540ACC2468
:1011B000DD2413C09F85953241F481E0C82ED12CE7
:1011C0006624762CEAE0E88B08C0B101FF858F2FFA
:1011D000992787FD90950E94540AF101838183FF2E
:1011E00004C0ED85FE85F49103C0ED85FE85F08198
:1011F000FF872F85222309F08BCDF101868197810E
:1012000062960FB6F894DEBF0FBECDBFDF91CF91CF
:101210001F910F91FF90EF90DF90CF90BF90AF9014
:101220009F908F907F906F905F904F903F902F9006
:1012300008950F931F93CF93DF93869F8001879F1D
:10124000100D969F100D1124C8010E943509EC0164
:10125000009729F0A80160E070E00E943F0ACE01EB
:10126000DF91CF911F910F910895CF93DF93AC0140
:10127000029710F442E050E020E030E0A0919A04A0
:10128000B0919B04BD01F901109709F44CC08D91F8
:101290009C9111978417950731F14817590738F435
:1012A0002115310519F08217930708F49C01FD01FF
:1012B000A281B381109759F721153105A1F1C90118
:1012C000841B950B049708F4A901DB01E0E0F0E032
:1012D000109749F18D919C91119782179307F9F41A
:1012E0004217530779F4ED018A819B81309719F0F9
:1012F0009383828304C090939B0480939A04CD01CE
:1013000002964AC0241B350BFD01E20FF31F4193E7
:101310005193225030402D933C93CF013DC0FD01AD
:10132000A281B381D5CF8091980490919904892BA3
:1013300041F4809125029091260290939904809324
:101340009804E0912302F0912402309741F4EDB724
:10135000FEB78091270290912802E81BF90BA0911B
:101360009804B09199049F012A1B3B0B2417350761
:1013700088F0CA0102962817390760F0CD01840F62
:10138000951F029690939904809398044D935D93D2
:10139000CD0102C080E090E0DF91CF910895CF931E
:1013A000DF93009709F454C0DC011297ED011B8212
:1013B0001A8280919A0490919B04009721F1FC017C
:1013C00040E050E0EA17FB0718F1ED01FB83EA83E8
:1013D0002D913C911197C20FD31FCE0102968E170B
:1013E0009F0771F48A819B81280F391F2E5F3F4F21
:1013F00011963C932E9382819381FD019383828386
:101400004115510559F4B0939B04A0939A0420C050
:10141000AF010280F381E02D3097A1F6EA01BB8392
:10142000AA83CA01029628813981820F931F8A17E5
:101430009B0771F48D919C911197280F391F2E5F96
:101440003F4F39832883FD01828193819B838A8367
:10145000DF91CF910895FC0105900020E9F7809578
:1014600090958E0F9F1F0895FC010590615070406C
:101470000110D8F7809590958E0F9F1F0895DC017D
:1014800040FF03C001C06D936D9342505040D8F7A8
:101490000895FC016150704001900110D8F78095CB
:1014A00090958E0F9F1F08950F931F93CF93DF93F7
:1014B0008C01EB018B81992781FF1CC082FF0DC03D
:1014C0002E813F818C819D812817390764F4E88142
:1014D000F9810193F983E88306C0E885F985802FB7
:1014E0000995892B39F48E819F8101969F838E8384
:1014F000C80102C08FEF9FEFDF91CF911F910F9135
:101500000895629FD001739FF001829FE00DF11D4D
:10151000649FE00DF11D929FF00D839FF00D749F6D
:10152000F00D659FF00D9927729FB00DE11DF91F19
:10153000639FB00DE11DF91FBD01CF011124089576
:10154000A1E21A2EAA1BBB1BFD010DC0AA1FBB1FC7
:10155000EE1FFF1FA217B307E407F50720F0A21B39
:10156000B30BE40BF50B661F771F881F991F1A94A6
:1015700069F760957095809590959B01AC01BD01D0
:10158000CF0108958F931CD08F9109F08062089548
:101590001FD001921A94E1F70895E199FECFBFBBE5
:1015A000AEBB0DBA11960FB6F894E29AE19A0FBE4F
:1015B0000895F3DF012CF1DF1124089585FD10C09B
:1015C000806291110DC08136ECF38B37DCF7089502
:1015D000E199FECFBFBBAEBBE09A11960DB2089564
:0615E000992788270895F9
:1015E6002A2A2A2A2A002A2A2A2A2A2054616368B1
:1015F6006F6D657465722F4D6F746F7220436F6ED9
:1016060074726F6C6C65722070726F6772616D00B8
:101616004379636C65732F526563203D2025640A08
:10162600006F637232202020202020203D20256478
:101636000A002F2D5C7C002563204144433A202577
:10164600303278202530327820544F503A202530D9
:1016560034782050574D3A202530346C782050434A
:10166600543A2025336C6420456E61626C653A25D8
:10167600640D0052504D3A206E6F207369676E619B
:101686006C0D0052504D3A2025356C6420202020E8
:10169600200D0064656C746154696D65203D2025DC
:1016A6006C640A000A4379636C65732F5265762071
:1016B6003D2025640A00456E746572206E657720AC
:1016C6006379636C65732F7265763A20000A446904
:1016D6007361626C65204D6F746F72000A456E61AE
:1016E600626C65204D6F746F72000A4F4352322050
:1016F6003D2025640A00456E746572204F435232C0
:0A1706003A200000009C04200000BF
:00000001FF
